:020000040000FA
:0200000038289E
:08000800A000030E8312A10009
:10001000063081070B11C803C00B0F28C103A20BC8
:100020002028C830A2003A08031DBA03A30B2028D9
:100030000A30A3003F08031DBF033B08031DBB0399
:10004000210E8300A00E200E09002034203420341D
:100050007334733477342E34613473346D34203414
:10006000563431342E343634203420342034203485
:100070008316FF23900083128501831632309F0080
:1000800080308100FB30DF3985008312203084000E
:100090008001840A841F4828A20AA30AFF30810035
:1000A0008B168B1747212608C3002708C400391573
:1000B00039088500CB20051A5F28392237143911F9
:1000C00085018316A83099008312033099003718F0
:1000D000812A2408A504031DA82B3230B820031C54
:1000E000B7143430B820031C37151D212F0803190D
:1000F000B715BB00B71A8128B71981283B08031927
:100100008628CC20381A892837127A28851D371777
:100110008C28371A7A28B711B916E6212C0803194A
:100120009428BA002830AD202D0803199A28BA0067
:100130002A30AD20B912E6212E08BA002630AD20B3
:100140003716B71EA528B712A728851DB716371F63
:1001500076283713381E8C28762884000008C300C0
:10016000840A0008C400CC203A08031DB328080004
:1001700084003008800731080318013E840A800794
:100180000310800C8403800C300800023108031C2B
:10019000013E840A00020800E321B81038111D2135
:1001A0003818EC2832080E023308031C013E0F02F7
:1001B000B71CDD28031CB814DF280318B814340852
:1001C0000E023508031C013E0F02371DEA28031CEE
:1001D0003815EC28031838153808BC06BC1CF32861
:1001E0000530BE00FB283E080319FB28BE0BFB2888
:1001F0003812B81838163C1D00293608BF000929E6
:100200003608031909293F08031D0929B8123819AE
:10021000B8163C1C0E291430BD0016293D080319E0
:100220001629BD0B1629B8113818B8153808BC00A6
:10023000B819B715B81AB71508003810C001003042
:10024000C1003330C0008E018F0141309000432146
:10025000381808000E080F040319272943213818FD
:10026000080009300F0203183D29051E2E299001B0
:1002700003300F02031C232908004321381808000B
:10028000051E3D2923296400C11B381408002630AF
:10029000840000309621031D24142830840003308C
:1002A0009621031DA4142A30840006309621031DD4
:1002B00024152C30840009308A21031DA4152D300B
:1002C00084000B308A21031D24162E3084000D304B
:1002D0008A21031DA4162F3084000F308A21031DAC
:1002E00024173030840011309621031DA4173230BA
:1002F000840014309621031D2514343084001730F7
:100300009621031DA514363084001A308A21031D5E
:1003100025150800C200AB218000420AAB2100066F
:10032000FF3A03190800800103110800C200AB2145
:100330008000840AC20A4208AB218000420AAB2135
:1003400000068403000603190800DC308000840ADC
:1003500005308000080083169B001C141A088312C5
:100360000800C200C9210008CE21C20A840A42083E
:10037000C9210008CE21420AC921000884030006D1
:10038000CE29C200C9210008CE21420AC921000994
:10039000CE2983161C159B00831208008B1383162D
:1003A0009A0055309D00AA309D009C148312640071
:1003B0008C1FD7298C1383161A081C111C141A06BB
:1003C00083128B1708003908850008008316013056
:1003D0008506831208005F300E020530031C013EC3
:1003E0000F02031C451559300E020630031C013E56
:1003F0000F020318C515080045084A060C39031DED
:10040000102A4B0803190800CB0B080045190C2AC9
:10041000C5190E2AC516080045160800451708001C
:10042000CA060530CB008F30C5050800051E1F2AFF
:100430001B2A851D1F2AC70B0800C51408000A3097
:10044000C700C5100800E3216400C81F242A273014
:10045000C800C90B0800451408004511C511E32167
:100460001D21381CEB21FC21C81F08002830C807BB
:10047000292A0A30C700C510B91A432A0530C90015
:10048000B9164510472A0530C900B9124510162281
:10049000C5184E2A2322451C472A3C2AB91239087E
:1004A000850008000A30C700C510B91A5C2A05305B
:1004B000C900B9164510602A0530C900B9124510A7
:1004C0001922C518672A2322451C602A552AB91209
:1004D000390885001D210800B91A732A0530C900A2
:1004E000B9164510772A0530C900B91245102D22DA
:1004F000C51A7D2A451C772A6C2AB912390885004D
:1005000008000130CC000530CB0052226C224C3068
:1005100084000B30D822522237234618D02AC6181E
:10052000942A4619C02A872A0030C900B9164510F6
:100530000008C300840A0008C4002D22851DB62AC5
:100540004519AC2AC519A52A9D2AC30FA82AC40A91
:100550004408083C03189D2A0130C3020318013CDB
:10056000C4024408023C031C9D2AA52A44088000BA
:100570008403430880002608C3002708C400D22A49
:100580000030C900B91645102D22851DC82AC42A7D
:100590003818D22A0E088000840A0F088000D22A58
:1005A0006330D822B9123908850064235222872A81
:1005B000CE00D101CF01D00100080319E92ACD00F6
:1005C000D00A50080A3A031DE72ACF0AD001CD0B02
:1005D000E02A5118F32A51143230C900B9124510DB
:1005E0000130CD00112BD118002BD1144F08031965
:1005F000082BCD00CD070A30C900B9164510112BC4
:100600005119082B51151E30C900B9124510F02A96
:10061000D1015008031DF92A1E30C900B916451032
:10062000F02A2D22851D0800451A292B451B302B49
:10063000451C112BCD030319E92AB91A242B0A30C2
:10064000C900B9164510112B0A30C900B91245105E
:10065000112B80030009031D352B4E088000352B1C
:10066000800A00084E02031C80016C22D92AC601B0
:1006700003308A004C088207CB28482B4C2B4E2B8A
:10068000502B542B562B582B5A2B5E2B602B622B46
:1006900026308400C61408002830492B2A30492B04
:1006A0002C308400461408002D30512B2E30512B55
:1006B0002F30512B303084004615080032305B2B30
:1006C00034305B2B3630512B4C038207712B762B49
:1006D0007B2B802B852B8A2B8F2B942B992B9E2B5E
:1006E000A32B263084000030B1210800283084007C
:1006F0000330B12108002A3084000630B1210800FF
:100700002C3084000930C12108002D3084000B30CA
:10071000C12108002E3084000D30C12108002F3087
:1007200084000F30C1210800303084001130B12125
:100730000800323084001430B121080034308400C5
:100740001730B1210800363084001A30C12108006A
:100750000130C6230230C6230430C6230830C62326
:100760001030C6232030C6234030C6238030C62335
:100770000130C8230230C8230430C8233C30C900EC
:10078000B91245102322451CC22BA82B2405C92BC6
:100790002505031DD02B0A30C900B9164510D42BEE
:1007A0001E30C900B91645102322451CD42B0A302F
:0E07B000C900B91245102322451CDB2B08009E
:02400E00CC3FA5
:10420000DC000500D900DC000500D900D60006005E
:10421000D0000000FF000500FA000A00F50037009A
:10422000C800DC000500D900080007000F00B0003E
:084230000400B4000A00F500CF
:00000001FF
